:100000000C9446000C9463000C9463000C94630001
:100010000C9463000C9463000C9463000C946300D4
:100020000C9463000C9463000C9463000C946300C4
:100030000C9463000C9463000C9463000C946300B4
:100040000C9463000C9463000C9463000C946300A4
:100050000C9463000C9463000C9463000C94630094
:100060000C9463000C9463000C9463000C94630084
:100070000C9463000C9463000C9463000C94630074
:100080000C9463000C9463000C94630011241FBE55
:10009000CFEFD0E1DEBFCDBF11E0A0E0B1E0E4E101
:1000A000F3E000E00BBF02C007900D92A030B10753
:1000B000D9F711E0A0E0B1E001C01D92A030B10776
:1000C000E1F70C948A000C940000CF93DF93CDB736
:1000D000DEB710923B0080E480933A001092380023
:1000E00010923700109235001092340010923200B6
:1000F000109231001092230080E38093220010922E
:100100006200109261001092650010926400DF910D
:10011000CF910895C9EFD0E1DEBFCDBF0E94650049
:1001200081E090E09E838D838091390099278170D2
:100130009070009729F480913B00806480933B008D
:1001400080913900992782709070009709F06FC0F4
:1001500080913900992782709070009731F48FEB6D
:1001600090913B00892380933B008091390099272F
:1001700082709070009719F58AE090E09A838983E5
:1001800089819A810097D9F08091390099278270EE
:100190009070009771F480E395E79C838B838B814B
:1001A0009C81009731F08B819C8101979C838B838C
:1001B000F6CF89819A8101979A838983E1CF8091D3
:1001C0003900992782709070009729F480913B0044
:1001D000806480933B0080913900992782709070F1
:1001E000009709F0ADCF8AE090E09A8389838981F6
:1001F0009A81009709F4A4CF8091390099278270E1
:100200009070009771F480E395E79C838B838B81DA
:100210009C81009731F08B819C8101979C838B831B
:10022000F6CF89819A8101979A838983E0CF809163
:1002300039009927847090700097E1F48D819E8138
:1002400081709070009709F415C08091390099274A
:1002500080749070009739F08FEB90913B00892368
:1002600080933B0005C080913B00806480933B00FD
:100270001E821D82809139009927887090700097A6
:1002800059F59FED8091230089238061809323009D
:1002900088EE93E09A83898389819A81009731F06F
:1002A00089819A8101979A838983F6CF809123006F
:1002B000982F90628FEE89238093230088EE93E03D
:1002C0009A83898389819A810097A1F289819A8191
:1002D00001979A838983F6CF80913900992780719D
:1002E0009070009751F49FEB80913B00892380939D
:1002F0003B0080913B0080933B008091390099271F
:1003000084709070009709F40FCF81E090E09E8395
:040310008D830ACF00
:00000001FF
